:0200000480007A
:100000001717000013070700971700009387870151
:10001000832007003711000013014100B7F1FFFFF3
:100020009381810037F2FF7F1302C200B702008084
:100030009382020133812000B3813000338240007B
:10004000B3825000170300009713000017F8FFFF5A
:1000500097FEFF7F970F008033431300B3C3230045
:1000600033483800B3CE4E00B3CF5F0023A0670003
:1000700023A2770023A4070123A6D70123A8F70111
:1000800097180000938848F8171800001308C8FA5A
:10009000B710111193801011372122221301212250
:1000A000B737333393873733374E4444130E4E44B8
:1000B000375F5555130F5F5583A108003702008045
:1000C000B7F2FF7F9382420013038000B713000052
:1000D0009383C30037F4FFFF13040401338241000C
:1000E000B382510033836100B38371003384810094
:1000F0009700008017F1FF7F97070000171E000090
:1001000017FFFFFFB3C0400033415100B3C7670082
:10011000334E7E00334F8F00232018002322280007
:100120002324F8002326C8012328E801171900001A
:100130001309C9ED97180000938848F1832009003E
:10014000032149008321890017020000130242FFA6
:100150009707000093878701170F0000130F0F0404
:10016000970200009382C2FD1708000013080800E0
:10017000970F0000938F8F0233421200B3C72700FE
:10018000334F3F00B382124033482800B3CF3F00C3
:1001900023A0480023A2F80023A4E80123A65800C6
:1001A00023A8080123AAF80117150000130585E705
:1001B00097150000938505EB370610F01306C6F27D
:1001C0006306B5028326C5002320D600832685005A
:1001D0002320D600832645002320D6008326050051
:1001E0002320D600130505016FF09FFD370510F0A1
:1001F000130505F2232005000000000000000000A8
:0402000000000000FA
:1010000044000080F00000803C0100806801008006
:1010100098010080000000000000000000000000B7
:10102000FFFFFFFFFFFFFFFFFFFFFFFFFFFFFFFFD0
:10103000FFFFFFFFFFFFFFFFFFFFFFFFFFFFFFFFC0
:10104000FFFFFFFFFFFFFFFFFFFFFFFFFFFFFFFFB0
:10105000FFFFFFFFFFFFFFFFFFFFFFFFFFFFFFFFA0
:040000058000000077
:00000001FF
